:100000000C9465000C94E30D0C94100E0C948D0070
:100010000C948D000C948D000C948D000C94570D55
:100020000C948D000C948D000C948D000C948D001C
:100030000C948D000C948D000C948D000C948D000C
:100040000C94FA160C948D000C9404030C94350354
:100050000C948D000C948D000C948D000C948D00EC
:100060000C94551C0C948D00020000000024002705
:10007000002A0000000000250028002B00000000DE
:1000800000230026002900040404040404040402DC
:100090000202020202030303030303010204081025
:1000A00020408001020408102001020408102000F2
:1000B0000000070002010000030406000000000029
:1000C00000000000A10477056F1B11241FBECFEFB5
:1000D000D8E0DEBFCDBF12E0A0E0B1E0E8E5F2E598
:1000E00002C005900D92A03EB107D9F714E0A0EE32
:1000F000B2E001C01D92A039B107E1F710E0CAECEF
:10010000D0E004C02297FE010E945725C43CD107CD
:10011000C9F70E94DC000C942A290C940000CF93AC
:10012000DF9360ED77E080E090E00E948217C2E804
:10013000D3E0CE0160E071E00E94170660ED77E049
:1001400080E090E00E948217CE010E949C02DF9125
:10015000CF910895CF93DF9386E060E00E949F18CF
:10016000C2E8D3E0CE0140E056E960E070E00E94D2
:10017000BB03CE016BE071E00E941706CE0169E17E
:1001800071E00E941706CE0163E371E00E9417063A
:10019000CE0161E471E00E941706CE016FE471E0C8
:1001A0000E941706CE0160E671E00E9417060E94C9
:1001B0008F00DF91CF9108957F928F929F92AF929F
:1001C000BF92CF92DF92EF92FF920F931F93DF9334
:1001D000CF93CDB7DEB727970FB6F894DEBF0FBE2B
:1001E000CDBF0E94B31784E194E00E94161B85E006
:1001F00061E00E949F1885E060E00E94C3180E94A1
:10020000AA0082E060E00E949F1886E060E00E9401
:100210009F188CE061E00E949F188DE061E00E94D1
:100220009F188DE061E00E94C31885E061E00E94A4
:10023000C3188091EB02879588278795E090EC02A0
:10024000EE0CEE0CEE0CE82A8091ED02E82A80918B
:10025000EF028295880F807E0091F002000F000F60
:10026000000F082B8091EE02082B9091F1029795D8
:10027000992797958091F5028295807F892B90919F
:10028000F702892B9091F902990F990F990F982BEA
:10029000A090F402AA0CA92A9091F20297959927AE
:1002A00097958091F3028295880F880F807C892B27
:1002B0009091F802892BC090F602CC0CCC0CC82A85
:1002C00084E194E068EC70E00E94521B84E194E0C9
:1002D0006E2D0E94D61A84E194E0602F0E94D61AF7
:1002E00084E194E06A2D0E94D61A84E194E06C2D9A
:1002F0000E94D61A84E194E00E94551B0AEF10E098
:100300006E010894C11CD11CA4E0AA2EB12CAC0E25
:10031000BD1EF2E08F2E912C8C0E9D1E77247394BF
:1003200084E194E069EC70E00E94521B82E00E943C
:10033000FB18009709F0A1C0E1EEEE2EE2E0FE2EE0
:1003400084E194E00E944B1AF70181937F01FBEE58
:10035000EF16F2E0FF06A1F784E194E00E94551B3E
:100360008091E10289838091E30290E0A0E0B0E017
:10037000BA2FA92F982F88272091E40230E040E07F
:1003800050E0822B932BA42BB52B2091E20230E07E
:1003900040E050E02770307040705070A901332762
:1003A0002227822B932BA42BB52B8C839D83AE838A
:1003B000BF838091E602829586958695837090E052
:1003C0002091E50230E0220F331F220F331F822BD2
:1003D000932B9B838A8313C082E893E00E947A0266
:1003E000823029F0833031F0813049F406C00AEFC1
:1003F00010E005C002E310E002C008EE13E082E85E
:1004000093E00E944B021816190634F386E00E940E
:10041000FB182091E002009751F1222311F4709211
:10042000E00282E893E063E771E042E050E00E947E
:10043000860582E893E062E771E041E050E00E94C7
:10044000860582E893E0B60141E050E00E9486050F
:1004500082E893E0B50144E050E00E94860582E81E
:1004600093E0B40142E050E00E94860506C02223DA
:1004700021F00E948F001092E002B80180E090E02D
:100480000E9482178CE060E00E94C3188DE060E05B
:100490000E94C31845CFFC0184859585FC01E05C72
:1004A000FF4F208131818E5B9F4FFC0180819181C4
:1004B000281B390B2F733070C9010895FC01848506
:1004C0009585FC01E05CFF4F40815181FC01EE5BB2
:1004D000FF4F208131814217530741F00190F08195
:1004E000E02DE80FF91F208130E002C02FEF3FEF31
:1004F000C9010895FC0184859585FC01E05CFF4FEE
:1005000040815181FC01EE5BFF4F20813181421718
:10051000530771F0A081B181A80FB91F2C91808180
:10052000918101968F7390709183808330E002C037
:100530002FEF3FEFC9010895DC011E968D919C912C
:100540001F97FC01E05CFF4F8E5B9F4F4081518104
:10055000DC012D913C91119742175307B9F708958B
:100560001F93FC01162F26853785D901A05CBF4F4C
:100570008D919C91019660E470E00E94BA24D901AB
:10058000AE5BBF4F4D915C91119784179507D1F3E6
:10059000D901A05CBF4F0D90BC91A02DA20FB31F3D
:1005A0001C93A685B785A05CBF4F11969C938E9334
:1005B000A689B7892C9181E090E0058C02C0880F54
:1005C000991F0A94E2F7282B2C9381E090E01F9169
:1005D0000895FB01E05CFF4F208131812F5F3F4F89
:1005E0002F733070DB01AE5BBF4F4D915C91119763
:1005F0002417350739F0A081B181A60FB71F8C935E
:1006000031832083089508951F920F920FB60F92A1
:1006100011242F933F934F935F936F937F938F9307
:100620009F93AF93BF93EF93FF938091C6006AEFC0
:1006300072E00E94E902FF91EF91BF91AF919F910B
:100640008F917F916F915F914F913F912F910F907B
:100650000FBE0F901F90189582E893E00E944B0206
:10066000009711F00E94030308951F920F920FB696
:100670000F9211242F933F935F936F937F938F93E8
:100680009F93AF93BF93EF93FF9320917E0330919D
:100690007F0380918003909181032817390731F4FB
:1006A0008091C1008F7D8093C10016C0E0918003CE
:1006B000F0918103E25CFC4F208180918003909156
:1006C0008103019660E470E00E94BA249093810354
:1006D000809380032093C600FF91EF91BF91AF916B
:1006E0009F918F917F916F915F913F912F910F908B
:1006F0000FBE0F901F9018958F92AF92BF92CF921E
:10070000DF92EF92FF920F931F93DF93CF93CDB7BA
:10071000DEB7FC011382128288EE93E0A0E0B0E025
:1007200084839583A683B78389E791E0918380834F
:100730007587648757874687318B208B138B028B95
:10074000F58AE48AD78AC68AB18EA08E828E8E857B
:10075000838F8F85848F8889858F8989868FCF91B4
:10076000DF911F910F91FF90EF90DF90CF90BF909E
:10077000AF908F9008959F92AF92BF92CF92DF92E9
:10078000EF92FF920F931F93CF93DF93EC017A01C7
:100790008B0199249394EC89FD8981E090E00E8C83
:1007A00002C0880F991F0A94E2F7808360E874E81A
:1007B0008EE190E0A80197010E94CD2421503040A5
:1007C00040405040569547953795279590E4A92E7F
:1007D00092E4B92E9FE0C92ED12C12C09924EC8945
:1007E000FD891082C601B501A80197010E94CD24A0
:1007F00021503040404050405695479537952795B9
:1008000080E12030380710F0992041F7E889F98914
:100810003083EA89FB892083EE89FF89408181E06A
:1008200090E09C010A8C02C0220F331F0A94E2F769
:10083000422B4083EE89FF8940819C010B8C02C0D2
:10084000220F331F0A94E2F7422B4083EE89FF897F
:1008500040819C010C8C02C0220F331F0A94E2F7E6
:10086000422B4083EE89FF8920810D8C02C0880FC6
:10087000991F0A94E2F7809582238083DF91CF91BC
:100880001F910F91FF90EF90DF90CF90BF90AF90AE
:100890009F900895CF93DF93FC0186859785DC01B7
:1008A000A05CBF4F8E5B9F4F4D915C911197EC0107
:1008B0002881398142175307B9F7A689B7894C9126
:1008C00081E090E09C01028C02C0220F331F0A9449
:1008D000E2F7209524232C93A689B7894C919C019B
:1008E000038C02C0220F331F0A94E2F720952423C1
:1008F0002C93A689B7894C919C01048C02C0220FCD
:10090000331F0A94E2F7209524232C93A689B789F4
:100910002C91058C02C0880F991F0A94E2F78095EC
:1009200082238C9384859585FC01EE5BFF4F2081AB
:100930003181805C9F4FFC0131832083DF91CF9117
:100940000895109285031092840388EE93E0A0E04E
:10095000B0E08093860390938703A0938803B093BD
:100960008903E4E8F3E089E791E0929382938AEFC8
:1009700092E0958784878EE393E09787868785EC5E
:1009800090E0918B808B84EC90E0938B828B80EC59
:1009900090E0958B848B81EC90E0978B868B86EC36
:1009A00090E0918F808F84E0828F83E0838F87E057
:1009B000848F85E0858F81E0868F08958F929F9246
:1009C000AF92BF92CF92DF92EF92FF920F931F935D
:1009D000CF93DF934C017B0182E0A82EB12CA80CB1
:1009E000B91CC0E0D0E0CC24DD24F50161915F01A9
:1009F000C7014AE050E00E943B078C01C7016EE24C
:100A00000E941A06080F191FC00ED11E2196C3306E
:100A1000D10559F7C701F40165814AE050E00E9411
:100A20003B07C80ED91EC601DF91CF911F910F91D0
:100A3000FF90EF90DF90CF90BF90AF909F908F90FE
:100A40000895FC0189E991E09183808312821382E9
:100A50001482158208950F93FC0189E991E0918336
:100A6000808362834383248305830F910895FC016F
:100A700089E991E091838083428353836483758302
:100A80000895FC0189E991E091838083DB012D9138
:100A90003D914D915C911397228333834483558319
:100AA0000895CF93DF93FC01EB0188819981AA819E
:100AB000BB8182839383A483B583CF01DF91CF91E0
:100AC0000895FC01428353836483758308959B01D9
:100AD000BC016E5F7F4FC90144E050E00E94ED27EA
:100AE0009C0181E02115310509F080E0089589E934
:100AF00091E09093A2038093A1031092A30310921C
:100B0000A4031092A5031092A6030895CF92DF923A
:100B1000EF92FF920F931F93CF93DF936C017B01B2
:100B20008A01C0E0D0E00FC0D7016D917D01D601F0
:100B3000ED91FC910190F081E02DC6010995C80F5F
:100B4000D91F015010400115110571F7CE01DF9139
:100B5000CF911F910F91FF90EF90DF90CF9008956C
:100B6000DB010D900020E9F7AD0141505040461BDC
:100B7000570BDC01ED91FC910280F381E02D09958A
:100B80000895EF92FF920F931F93CF93DF937C0111
:100B9000062F172FC0E0D0E0F8010F5F1F4F6491C0
:100BA000662351F0F701A081B181ED91FC91C7015D
:100BB0000995C80FD91FF0CFCE01DF91CF911F91BA
:100BC0000F91FF90EF900895AF92BF92CF92DF9276
:100BD000EF92FF920F931F93CF93DF937C016B01F2
:100BE000C0E0D0E000E010E010C0D701ED91FC9132
:100BF000A080B180C601BE010E94B613682FC70154
:100C0000F5010995080F191F2196F6018481958138
:100C1000C817D90750F3C801DF91CF911F910F91E9
:100C2000FF90EF90DF90CF90BF90AF9008950E941B
:100C3000B0050895DC01ED91FC910190F081E02D6B
:100C4000099508959C01CB01DB01ED91FC91019088
:100C5000F081E02DB901099508950F931F93CF936B
:100C6000DF93EC016DE00E941A068C01CE016AE070
:100C70000E941A06080F191FC801DF91CF911F911A
:100C80000F9108950F931F93CF93DF93EC010E9470
:100C9000C1058C01CE010E942D06080F191FC80145
:100CA000DF91CF911F910F9108950F931F93CF93D1
:100CB000DF93EC010E94E4058C01CE010E942D0619
:100CC000080F191FC801DF91CF911F910F9108954F
:100CD0000F931F93CF93DF93EC010E94B0058C011B
:100CE000CE010E942D06080F191FC801DF91CF9178
:100CF0001F910F9108950F931F93CF93DF93EC01F2
:100D00000E941A068C01CE010E942D06080F191FA1
:100D1000C801DF91CF911F910F9108950F931F93F9
:100D2000CF93DF93EC010E9422068C01CE010E943A
:100D30002D06080F191FC801DF91CF911F910F9148
:100D400008958F929F92AF92BF92CF92DF92EF92CF
:100D5000FF920F931F93DF93CF93CDB7DEB7A19789
:100D60000FB6F894DEBF0FBECDBF6C01042FE52F88
:100D7000CB01122F19A2223008F41AE021E2E22E50
:100D8000F12CEC0EFD1E812E9924AA24BB2403C055
:100D9000022FE32FCA01602F7E2FA50194010E942C
:100DA000CD24129F802D1124081B0894E108F1081E
:100DB0000A3014F4005D01C0095CF70100832115BD
:100DC00031054105510521F7C601B7010E94B00563
:100DD000A1960FB6F894DEBF0FBECDBFCF91DF91C5
:100DE0001F910F91FF90EF90DF90CF90BF90AF9049
:100DF0009F908F9008952115310549F4DC01ED9104
:100E0000FC910190F081E02D642F099508950E94D6
:100E1000A10608950F931F93CF93DF93EC010E94D7
:100E2000FB068C01CE010E942D06080F191FC80178
:100E3000DF91CF911F910F9108959A01AB0160E06E
:100E400070E00E94FB0608950F931F93CF93DF93EA
:100E5000EC019A01AB0160E070E00E94FB068C019E
:100E6000CE010E942D06080F191FC801DF91CF91F6
:100E70001F910F9108959A01462F50E060E070E0B5
:100E80000E94FB0608950F931F93CF93DF93EC010D
:100E90009A01462F50E060E070E00E94FB068C0152
:100EA000CE010E942D06080F191FC801DF91CF91B6
:100EB0001F910F910895CF92DF92EF92FF920F93BF
:100EC0001F93CF93DF93EC017A018B01211531053C
:100ED00041F4E881F9810190F081E02D642F0995BA
:100EE0001AC02A303105A9F477FF12C06DE20E94C2
:100EF0001A066C0144275527BA014E195F09600B89
:100F0000710BCE012AE00E94A106C80ED91E04C0B2
:100F10002AE00E94A1066C01C601DF91CF911F91CA
:100F20000F91FF90EF90DF90CF9008950F931F9354
:100F3000CF93DF93EC010E945B078C01CE010E94EE
:100F40002D06080F191FC801DF91CF911F910F9136
:100F500008959A01FB01AF01662757FD6095762F32
:100F60000E945B0708950F931F93CF93DF93EC01CB
:100F70009A01CB01AC01662757FD6095762FCE0113
:100F80000E945B078C01CE010E942D06080F191FDD
:100F9000C801DF91CF911F910F9108956F927F92B9
:100FA0009F92AF92BF92CF92DF92EF92FF920F93F8
:100FB0001F93CF93DF933C017A018B01C22ECB01AB
:100FC000BA0120E030E0A9010E94572187FF0AC042
:100FD000C3016DE20E941A06EC0117FB109517F988
:100FE000109502C0C0E0D0E0DD2450E040E030E0E9
:100FF0002FE311C0DA01F9016B2F742F8F2F922F7D
:1010000020E030E040E251E40E947920562F472F43
:10101000382F292FD394DC1468F3C801B701DA0103
:10102000F9012B2F342F4F2F5E2F0E94211F5B01C0
:10103000F82E992E7B2D0E94AB1D162FD72EE82E51
:10104000092F0E9439229B01AC016A2D7B2D8F2D27
:10105000992D0E944E1F962EA72EB82EF92EC30151
:10106000412F5D2D6E2D702F2AE030E00E94FB068F
:10107000C80FD91FCC20B9F1C30161EA71E00E9409
:10108000B005C80FD91F2FC0692D7A2D8B2D9F2D2C
:1010900020E030E040E251E40E947F1FD62EB72EC0
:1010A000A82E992E0E94E7217B010027F7FC0095CE
:1010B000102FC301B801A7012AE030E00E945B07AE
:1010C000C80FD91FC801B7010E9487219B01AC013D
:1010D0006D2D7B2D8A2D992D0E944E1F962EA72EA9
:1010E000B82EF92ECA94CC2079F6CE01DF91CF919B
:1010F0001F910F91FF90EF90DF90CF90BF90AF9036
:101100009F907F906F9008950E94CE0708950F934F
:101110001F93CF93DF93EC010E94CE078C01CE0189
:101120000E942D06080F191FC801DF91CF911F9152
:101130000F910895CF93DF93EC010E944E176887BB
:1011400079878A879B87E881F9810680F781E02D7E
:10115000CE0109959C0197FF15C00E944E17288566
:1011600039854A855B85621B730B840B950B2C813B
:101170003D814E815F81621773078407950718F3DD
:101180002FEF3FEFC901DF91CF910895CF93DF9308
:10119000EC010E944E17688779878A879B87E881D0
:1011A000F9810084F185E02DCE0109959C0197FF1E
:1011B00015C00E944E17288539854A855B85621BBC
:1011C000730B840B950B2C813D814E815F816217DF
:1011D00073078407950718F32FEF3FEFC901DF91DD
:1011E000CF910895CF93DF93EC01CE010E94C60802
:1011F0009C0197FD0FC08D32910561F0C0978A3038
:10120000910540F0E881F9810680F781E02DCE015B
:101210000995EBCFC901DF91CF910895FC0144837B
:1012200055836683778308956F927F928F929F9202
:10123000AF92BF92CF92DF92EF92FF920F931F93E4
:10124000CF93DF933C016B014A0159017801FB0107
:101250008081882391F1C0E0D0E000E010E026C05A
:10126000F601E00FF11F2081332727FD309582170B
:10127000930731F40F5F1F4F0815190518F01DC0B3
:1012800000E010E0E114F10479F0F501EC0FFD1F2E
:101290002081332727FD30958217930729F4219663
:1012A000CE15DF0518F00BC0C0E0D0E0C3010E94EE
:1012B0009A0818161906A4F202C081E001C080E065
:1012C000DF91CF911F910F91FF90EF90DF90CF9022
:1012D000BF90AF909F908F907F906F9008950F93E5
:1012E0001F93CF93DF939A01FB0101900020E9F750
:1012F0003197E61BF70BEA0109900020E9F78E0110
:1013000001501040041B150BAF010E941409DF911E
:10131000CF911F910F91089540E050E00E946F0916
:1013200008950F931F9320E030E000E010E00E944A
:1013300014091F910F9108959F92AF92BF92CF927F
:10134000DF92EF92FF920F931F93CF93DF936C0185
:10135000A62E0E94F208EC0197FD4EC0EE24FF2459
:1013600087019924BB24A7FCB094CA15DB0531F191
:10137000CD32D10509F1CE01C0978A309105F0F444
:10138000C801B7012AE030E040E050E00E949B2411
:101390007B018C01CE01AA2797FDA095BA2FE80EFC
:1013A000F91E0A1F1B1F80ED9FEFAFEFBFEFE80E86
:1013B000F91E0A1F1B1F02C099249394D601ED91B8
:1013C000FC910680F781E02DC6010995C6010E94B7
:1013D000C608EC01C0978A30910538F2CA15DB05C2
:1013E00021F2992061F010950095F094E094E11CB1
:1013F000F11C011D111D03C0EE24FF248701B7015C
:10140000C801DF91CF911F910F91FF90EF90DF9076
:10141000CF90BF90AF909F90089561E00E949C098B
:1014200008956F927F928F929F92AF92BF92CF92C8
:10143000DF92EF92FF920F931F93CF93DF93EC0114
:10144000762E0E94F208D82E87FD7DC0BB24AA24E8
:1014500090E8992E8FE3882EEE24FF248701CC2478
:101460006624D714E1F18D2D8D32A1F18E32A9F1D0
:1014700080538A30A0F5C801B7012AE030E040E08F
:1014800050E00E949B247B018C018D2D992787FDC4
:101490009095A92FB92FE80EF91E0A1F1B1F80ED8A
:1014A0009FEFAFEFBFEFE80EF91E0A1F1B1FCC2006
:1014B000B1F0A5019401652F7A2D832F982D2DEC85
:1014C0003CEC4CEC5DE30E947F1FB62EA72E982EBD
:1014D000892E05C06624639402C0CC24C394E8819D
:1014E000F9810680F781E02DCE010995CE010E9499
:1014F000C608D82E982F90539A3008F4B2CF8E3267
:1015000009F4AFCF871509F4ACCF662041F01095F0
:101510000095F094E094E11CF11C011D111DCC20FC
:1015200069F0C801B7010E948721D501F4012B2F72
:101530003A2D4F2F582D0E947F1F09C0C801B701B7
:101540000E94872104C060E070E080E090E0DF91BD
:10155000CF911F910F91FF90EF90DF90CF90BF90B0
:10156000AF909F908F907F906F90089561E00E9460
:10157000110A0895CF92DF92EF92FF920F931F937B
:10158000CF93DF936C01EB017A0100E010E008C01B
:10159000C6010E949A0897FD06C089930F5F1F4FEE
:1015A0000E151F05A8F3C801DF91CF911F910F9170
:1015B000FF90EF90DF90CF900895AF92BF92CF92BF
:1015C000DF92EF92FF920F931F93CF93DF935C0113
:1015D000EA01790121153105B1F000E010E0C62ED5
:1015E000DD24C7FCD0940BC0C5010E949A0897FD6A
:1015F0000CC08C159D0549F089930F5F1F4F0E1588
:101600001F0590F302C000E010E0C801DF91CF9108
:101610001F910F91FF90EF90DF90CF90BF90AF9010
:1016200008952F923F924F925F926F927F928F9286
:101630009F92AF92BF92DF92EF92FF920F931F9310
:10164000DF93CF9300D000D0CDB7DEB71B01298345
:101650003A834B835C839091AB01981721F09F3FB5
:1016600009F0D8C104C0E8E6F0E0D4907DC08093D2
:10167000AB01E8E6F0E0D4909D2D9F3F09F4CAC18C
:10168000913031F1923009F449C0DD2009F06CC08D
:1016900014BC15BC94B5926094BD95B5916095BD90
:1016A000282F30E0F901E957FF4FE491F0E0EE0F09
:1016B000FF1FED58FF4F459154914093AB0350935A
:1016C000AC0325563F4FF90124912093AD034EC042
:1016D0001092800010928100909181009860909308
:1016E000810090918100916090938100282F30E0DB
:1016F000F901E957FF4FE491F0E0EE0FFF1FED58BD
:10170000FF4F459154914093B2035093B303255634
:101710003F4FF90124912093B40328C01092B000E8
:101720001092B1009091B00092609093B0009091AF
:10173000B10091609093B100282F30E0F901E95792
:10174000FF4FE491F0E0EE0FFF1FED58FF4F459182
:1017500054914093B9035093BA0325563F4FF90172
:1017600024912093BB0302C0D7FC54C161E00E94C6
:101770009F18DD2021F0FD2DF23009F0C1C041019C
:10178000AA24BB2460E079E08DE390E0A5019401F8
:101790000E94CD2429013A0179018A010894E108C7
:1017A000F108010911098FEFE816F104010511058F
:1017B00009F008F498C060E271EA87E090E0A501C2
:1017C00094010E94CD2479018A010894E108F1086E
:1017D000010911099D2D9230C9F4AFEFEA16F10409
:1017E0000105110509F008F485C068E478EE81E090
:1017F00090E0A50194010E94CD2479018A0108940A
:10180000E108F1080109110983E001C082E0BFEF9E
:10181000EB16F1040105110509F008F465C064E256
:1018200074EF80E090E0A50194010E94CD2479013D
:101830008A010894E108F10801091109DD20E1F0AD
:10184000ED2DE230D9F4FFEFEF16F104010511059B
:1018500009F008F451C062E17AE780E090E0A50168
:1018600094010E94CD2479018A010894E108F108CD
:101870000109110985E003C083E001C084E09FEF06
:10188000E916F1040105110579F170F169E07DE3D4
:1018900080E090E0A50194010E94CD2479018A01A5
:1018A0000894E108F10801091109DD2011F484E030
:1018B00001C086E0AFEFEA16F10401051105A1F0C1
:1018C00098F0830172019AE016950795F794E794D2
:1018D0009A95D1F70894E108F10801091109DD2072
:1018E00031F087E00AC081E0DD2011F006C085E01C
:1018F00085BD3CC082E001C084E08093B10036C069
:101900004101AA24BB2460E079E08DE390E0A501C9
:1019100094010E94CD2479018A010894E108F1081C
:1019200001091109B0E0EB16B0E0FB06B1E00B07CE
:10193000B0E01B0788F064E274EF80E090E0A5015E
:1019400094010E94CD2479018A010894E108F108EC
:101950000109110993E001C091E0ED2DE13031F46E
:1019600080918100887F892B8093810089819A8171
:10197000AB81BC810097A105B10591F0B101660F63
:10198000771F80E090E029813A814B815C810E9441
:101990009B2428EE33E040E050E00E94CD2403C0B9
:1019A0002FEF3FEFA9019D2D913099F0923019F161
:1019B000DD2081F5E7BC2093A7033093A803409373
:1019C000A9035093AA0380916E00826080936E00F9
:1019D00021C0F0928900E09288002093AE033093FA
:1019E000AF034093B0035093B10380916F008260C6
:1019F00080936F000FC0E092B3002093B503309343
:101A0000B6034093B7035093B8038091700082608F
:101A1000809370000F900F900F900F90CF91DF91F7
:101A20001F910F91FF90EF90DF90BF90AF909F902C
:101A30008F907F906F905F904F903F902F90089580
:101A4000813041F0813018F08230D1F409C0109219
:101A50006E00089580916F008D7F80936F000895D0
:101A6000809170008D7F8093700081E08093B00042
:101A70008091B100887F84608093B1001092B300A0
:101A800008951F93182F8091AB01811739F4E8E670
:101A9000F0E084919FEF9093AB0101C08FEF0E9423
:101AA000200D812F60E00E94C3181F9108951F929E
:101AB0000F920FB60F9211242F933F934F935F9382
:101AC0006F937F938F939F93AF93BF93EF93FF9306
:101AD0008091B5039091B603A091B703B091B8037C
:101AE0000097A105B10551F1E091B903F091BA0356
:101AF00080819091BB03892780838091B503909169
:101B0000B603A091B703B091B803181619061A06C8
:101B10001B06C4F48091B5039091B603A091B7035E
:101B2000B091B8030197A109B1098093B5039093CF
:101B3000B603A093B703B093B80304C08091AB0180
:101B40000E94410DFF91EF91BF91AF919F918F91B5
:101B50007F916F915F914F913F912F910F900FBEA9
:101B60000F901F9018958230E8F4E82FF0E0EE0F08
:101B7000FF1FE454FC4F71836083813041F08091FA
:101B800069008C7F842B80936900E89A0895809186
:101B90006900440F551F440F551F837F842B80938A
:101BA0006900E99A0895823068F4813011F0E8986C
:101BB00001C0E998E82FF0E0EE0FFF1FE454FC4F5E
:101BC0001182108208951F920F920FB60F92112466
:101BD0002F933F934F935F936F937F938F939F9335
:101BE000AF93BF93EF93FF938091BC039091BD039C
:101BF000009729F0E091BC03F091BD030995FF9196
:101C0000EF91BF91AF919F918F917F916F915F9174
:101C10004F913F912F910F900FBE0F901F901895ED
:101C20001F920F920FB60F9211242F933F934F9351
:101C30005F936F937F938F939F93AF93BF93EF9334
:101C4000FF938091BE039091BF03009729F0E0912C
:101C5000BE03F091BF030995FF91EF91BF91AF9142
:101C60009F918F917F916F915F914F913F912F91B4
:101C70000F900FBE0F901F901895009729F0BC0190
:101C800080E090E00E94DA260895EF92FF920F9391
:101C90001F937B018C01611571058105910549F048
:101CA0000E94D526A80197010E94EF249B01AC0158
:101CB00003C020E030E0A901B901CA011F910F91D2
:101CC000FF90EF900895EF92FF920F931F937B0187
:101CD0008C01621773078407950764F4CA01B90180
:101CE0006E197F09800B910B0E94450EE60EF71EC0
:101CF000081F191FB701C8011F910F91FF90EF90A6
:101D000008952F923F924F925F926F927F928F929F
:101D10009F92AF92BF92CF92DF92EF92FF920F937A
:101D20001F93DF93CF93CDB7DEB73B014C01190171
:101D30002A016D897E898F89988D6A197B098C09A2
:101D40009D09621A730A840A950AA40193010E94EC
:101D50009B24E218F30804091509A80197010E94C1
:101D6000EF242A0D3B1D4C1D5D1DB901CA01CF9109
:101D7000DF911F910F91FF90EF90DF90CF90BF9078
:101D8000AF909F908F907F906F905F904F903F901B
:101D90002F900895089570E0382F20E0622B732B68
:101DA000CB010895FC01808191810E94F525089561
:101DB000CF93DF93EC0188819981009711F00E9405
:101DC000F525198218821D821C821B821A82DF91DE
:101DD000CF9108950F931F93CF93DF93EC018B0165
:101DE0006F5F7F4F888199810E94E326009731F0D1
:101DF000998388831B830A8381E001C080E0DF919F
:101E0000CF911F910F910895CF93DF93EC018881BB
:101E10009981009729F08A819B818617970778F42A
:101E2000CE010E94EA0E882341F08C819D810097AB
:101E300031F4E881F981108202C080E001C081E0C4
:101E4000DF91CF910895EF92FF920F931F93CF935D
:101E5000DF93EC017B018A01BA010E94040F882301
:101E600021F4CE010E94D80E07C01D830C83888107
:101E70009981B7010E942928CE01DF91CF911F914E
:101E80000F91FF90EF900895CF93DF93FC011182A3
:101E900010821382128215821482168261157105D6
:101EA00059F0EB0109900020E9F7AE014150504094
:101EB000461B570B0E94230FDF91CF910895EF929D
:101EC000FF92CF93DF93EC01FB018617970761F038
:101ED000608171816115710529F0448155810E94ED
:101EE000230F02C00E94D80ECE01DF91CF91FF9048
:101EF000EF900895FC0111821082138212821582E4
:101F0000148216820E945F0F08950F931F938C0115
:101F10006115710561F0DB010D900020E9F7AD015D
:101F200041505040461B570B0E94230F02C00E9495
:101F3000D80EC8011F910F910895EF92FF920F9351
:101F40001F93DF93CF93CDB7DEB7A1970FB6F89469
:101F5000DEBF0FBECDBF7C01CB01BA01F7011182FC
:101F60001082138212821582148216828E010F5FF4
:101F70001F4FA80130E00E94DC28C701B8010E9471
:101F8000850FA1960FB6F894DEBF0FBECDBFCF91DF
:101F9000DF911F910F91FF90EF900895EF92FF92C4
:101FA0000F931F93DF93CF93CDB7DEB7A2970FB6F2
:101FB000F894DEBF0FBECDBF7C01CB01BA01F701A3
:101FC00011821082138212821582148216828E016F
:101FD0000F5F1F4FA80130E00E949328C701B8018E
:101FE0000E94850FA2960FB6F894DEBF0FBECDBF3C
:101FF000CF91DF911F910F91FF90EF900895EF9295
:10200000FF920F931F93DF93CF93CDB7DEB7619706
:102010000FB6F894DEBF0FBECDBF7C01CB01F70138
:1020200011821082138212821582148216828E010E
:102030000F5F1F4FB80150E00E940129C701B8018E
:102040000E94850F61960FB6F894DEBF0FBECDBF1C
:10205000CF91DF911F910F91FF90EF900895EF9234
:10206000FF920F931F93DF93CF93CDB7DEB76297A5
:102070000FB6F894DEBF0FBECDBF7C01CB01F701D8
:1020800011821082138212821582148216828E01AE
:102090000F5F1F4FB80150E00E947228C701B801BE
:1020A0000E94850F62960FB6F894DEBF0FBECDBFBB
:1020B000CF91DF911F910F91FF90EF900895EF92D4
:1020C000FF920F931F93DF93CF93CDB7DEB729977E
:1020D0000FB6F894DEBF0FBECDBF7C01862FF7018F
:1020E000118210821382128215821482168290E06D
:1020F0008E010F5F1F4FB80150E00E940129C701F8
:10210000B8010E94850F29960FB6F894DEBF0FBE66
:10211000CDBFCF91DF911F910F91FF90EF90089568
:10212000DF93CF9300D0CDB7DEB7FC0111821082D0
:102130001382128215821482168269831A82BE016A
:102140006F5F7F4F0E94850F0F900F90CF91DF91AF
:102150000895EF92FF920F931F93CF93DF93EC01BB
:102160007B010C811D8161157105B9F04115510587
:1021700091F0040F151FB8010E94040F882369F025
:10218000288139818C819D81820F931FB7010E9424
:1021900029281D830C8381E001C080E0DF91CF916D
:1021A0001F910F91FF90EF900895FB016081718165
:1021B000448155810E94A91008956115710561F04F
:1021C000DB010D900020E9F7AD0141505040461B66
:1021D000570B0E94A910089580E00895DF93CF93D4
:1021E00000D0CDB7DEB769831A82BE016F5F7F4F23
:1021F00041E050E00E94A9100F900F90CF91DF9125
:102200000895EF92FF920F931F93DF93CF9300D027
:1022100000D0CDB7DEB77C01862F90E08E010F5F36
:102220001F4FB8014AE050E00E947228F801019067
:102230000020E9F7AF0141505040401B510BC7014E
:10224000B8010E94A9100F900F900F900F90CF919E
:10225000DF911F910F91FF90EF900895EF92FF9201
:102260000F931F93DF93CF93CDB7DEB727970FB6AA
:10227000F894DEBF0FBECDBF7C01CB018E010F5F96
:102280001F4FB8014AE050E00E947228F801019007
:102290000020E9F7AF0141505040401B510BC701EE
:1022A000B8010E94A91027960FB6F894DEBF0FBEA2
:1022B000CDBFCF91DF911F910F91FF90EF900895C7
:1022C000EF92FF920F931F93DF93CF9300D000D034
:1022D00000D0CDB7DEB77C01CB018E010F5F1F4F61
:1022E000B8014AE050E00E940129F8010190002065
:1022F000E9F7AF0141505040401B510BC701B801F5
:102300000E94A91026960FB6F894DEBF0FBECDBF6F
:10231000CF91DF911F910F91FF90EF900895EF9271
:10232000FF920F931F93DF93CF93CDB7DEB72C9718
:102330000FB6F894DEBF0FBECDBF7C01CB01BA0152
:102340008E010F5F1F4FA8012AE030E00E94932802
:10235000F80101900020E9F7AF0141505040401BC7
:10236000510BC701B8010E94A9102C960FB6F89422
:10237000DEBF0FBECDBFCF91DF911F910F91FF90B8
:10238000EF900895EF92FF920F931F93DF93CF93F7
:10239000CDB7DEB72B970FB6F894DEBF0FBECDBF1B
:1023A0007C01CB01BA018E010F5F1F4FA8012AE00B
:1023B00030E00E94DC28F80101900020E9F7AF012D
:1023C00041505040401B510BC701B8010E94A91059
:1023D0002B960FB6F894DEBF0FBECDBFCF91DF9125
:1023E0001F910F91FF90EF9008950F931F938C0111
:1023F000FB0160817181448155810E94A91088236D
:1024000019F4C8010E94D80EC8011F910F910895B8
:102410000F931F938C016115710569F0DB010D901D
:102420000020E9F7AD0141505040461B570B0E9478
:10243000A910882319F4C8010E94D80EC8011F9161
:102440000F9108950F931F938C010E94EE10882323
:1024500019F4C8010E94D80EC8011F910F91089568
:102460000F931F938C010E940111882319F4C80156
:102470000E94D80EC8011F910F9108950F931F93CA
:102480008C010E942E11882319F4C8010E94D80ED5
:10249000C8011F910F9108950F931F938C010E9403
:1024A0006011882319F4C8010E94D80EC8011F9139
:1024B0000F9108950F931F938C010E948F11882311
:1024C00019F4C8010E94D80EC8011F910F910895F8
:1024D0000F931F938C010E94C211882319F4C80125
:1024E0000E94D80EC8011F910F910895CF93DF93DA
:1024F000FC01DB0180819181009731F06D917C912D
:10250000119761157105E9F4CD91DC911197209730
:1025100069F014962D913C9115972115310531F0F4
:10252000288130E0309521953F4F12C0009771F01F
:10253000248135812115310549F0FC01208130E0ED
:1025400007C00E942028282F392F02C020E030E049
:10255000C901DF91CF910895FC0144815581FB01B0
:10256000248135814217530729F40E94761221E015
:10257000009709F020E0822F0895FC018481958165
:10258000009741F46115710519F081E0FB0109C064
:1025900081E008950190F081E02D6115710531F41D
:1025A00081E09081992359F080E00895CF010E9445
:1025B00020289C0181E02115310509F080E0089573
:1025C0000E947612892F881F8827881F08950E94ED
:1025D000761221E0181619060CF020E0822F0895DB
:1025E0000E94761221E0181619060CF420E0822FC2
:1025F00008950E947612892F8095881F8827881F4A
:102600000895EF92FF920F931F93CF93DF93FC01F6
:10261000DB018617970729F18481958114962D9106
:102620003C91159782179307F1F40097D1F0008140
:102630001181CD91DC9111970FC0992787FD90955D
:102640000E94DD277C018991992787FD90950E9442
:10265000DD27E816F90639F4F80181918F01882306
:1026600061F781E001C080E0DF91CF911F910F9170
:10267000FF90EF900895FC01DB01CA0114964D9183
:102680005C91159724813581241B350B2817390758
:10269000A0F0208131812115310579F06D917C9177
:1026A00011976115710559F0820F931F0E94302810
:1026B0009C0181E02115310519F080E0089580E04A
:1026C0000895FC0144815581FB0124813581421725
:1026D000530728F040E050E00E943B13089580E04B
:1026E0000895FC01DB018481958114964D915C91E4
:1026F000159784179507B0F0208131812115310598
:1027000089F06D917C9111976115710569F0841BB9
:10271000950B820F931F0E9420289C0181E02115B8
:10272000310519F080E0089580E00895FC0184816E
:1027300095816817790730F40190F081E02DE60F5C
:10274000F71F40830895FC018481958168177907FC
:1027500020F480819181009729F41092C00360ECED
:1027600073E002C0680F791FCB010895FC018481DA
:1027700095816817790748F480819181009739F035
:10278000680F791FFB018081089580E0089580E043
:1027900008950E94B61308950F931F93CF93DF936C
:1027A000FC018B0141155105F1F061157105D9F05E
:1027B000C481D5812C173D0718F0FB01108213C08E
:1027C00041505040C21BD30B4C175D0708F4EA017F
:1027D00060817181620F731FC801AE010E943E28A3
:1027E000C00FD11F1882DF91CF911F910F910895D3
:1027F000CF93DF93FC01CA0124813581421753072F
:1028000078F4C081D181772767FD70958C0F9D1F6B
:102810000E941528009721F09C012C1B3D0B02C043
:102820002FEF3FEFC901DF91CF91089540E050E0D5
:102830000E94F8130895CF93DF93FC01CA0124810D
:1028400035814217530778F4C081D181FB01608143
:1028500071818C0F9D1F0E945828009721F09C01C8
:102860002C1B3D0B02C02FEF3FEFC901DF91CF9131
:10287000089540E050E00E941B140895DF92EF920B
:10288000FF920F931F93CF93DF93EC018C819D8177
:1028900048175907F8F47A010894E11CF11CE88103
:1028A000F981EE0DFF1DD0801082088119817727F4
:1028B00067FD7095C8010E944D280E0D1F1DF8017F
:1028C000D082009739F028813981AC01421B530B2B
:1028D0009A0102C02FEF3FEFC901DF91CF911F9105
:1028E0000F91FF90EF90DF900895FC014481558196
:1028F000415050400E943E140895AF92BF92CF9233
:10290000DF92EF92FF920F931F93CF93DF93FC011F
:102910006B018A01DB0114962D913C9115972115CD
:10292000310551F184819581009731F18217930728
:1029300018F14817590718F08C0101501040E08039
:10294000F180C701CFEFDFEF5701A00EB11E10C01D
:10295000F601608171810E945828009779F09C01EE
:102960002E193F090217130708F49E010196E90189
:10297000A816B90668F702C0CFEFDFEFCE01DF91EE
:10298000CF911F910F91FF90EF90DF90CF90BF906C
:10299000AF900895FC0144815581FB01248135816C
:1029A000421B530B0E947D140895AF92BF92CF92A9
:1029B000DF92EF92FF920F931F93CF93DF93F82E46
:1029C000E92E6B018A01E9012417350748F4342FF9
:1029D000212F8E01C901A92EE5015E01B22EE5016C
:1029E0008F2D9E2D6CEA71E00E94440FD601149643
:1029F0008D919C91159780179107D8F08C179D07A2
:102A000008F4EC01D601ED91FC911197EC0FFD1F3C
:102A1000B08010826D917C91600F711F8F2D9E2D63
:102A20000E94850FD601ED91FC911197EC0FFD1FCF
:102A3000B0828F2D9E2DDF91CF911F910F91FF902E
:102A4000EF90DF90CF90BF90AF900895CF93DF933A
:102A5000EC01FB01248135810E94D514CE01DF9168
:102A6000CF910895DC01ED91FC911197309729F4F5
:102A70000895861709F44083319680818823C9F729
:102A800008952F923F924F925F926F927F928F9212
:102A90009F92AF92BF92CF92DF92EF92FF920F93ED
:102AA0001F93CF93DF937C012B016A01DC01149605
:102AB0006D907C9015976114710409F4D9C0FB01E5
:102AC000848095808114910409F4D2C0DA011496AF
:102AD000AD90BC901597A818B908FC010081118130
:102AE000A114B104F1F413C0D6016C9111967C913C
:102AF000119714964D915C911597CE010E94FA277B
:102B0000D60114960D911C9115970C0F1D1FF20103
:102B100060817181C8010E945828EC01009721F75B
:102B2000A7C0B7FC02C0E30142C048012DC0E301C9
:102B3000C01BD10BC401B801AE010E94FA27C80D19
:102B4000D91DD6016C9111967C91119714964D91D7
:102B50005C911597CE010E94FA27D60114968D90AC
:102B60009C9015978C0E9D1EF20104811581060D17
:102B7000171DD70114968D919C9115978A0D9B1D59
:102B800015969C938E931497F20160817181C80110
:102B90000E9458283C01009751F6C401B8010E94D8
:102BA000292866C08C01080D191DCA0DDB1DD20134
:102BB0006D917C91C8010E945828009799F7C6151D
:102BC000D70509F455C0F701828193818C179D07C1
:102BD00008F045C0C701BE010E94EA0E882309F42F
:102BE00047C03DC0C701B201A9010E947D14EC019C
:102BF00097FD3EC0D7016D917C911197F2018481C0
:102C000095818C0F9D1F680F791F14964D915C91D3
:102C10001597481B590BCB018A0D9B1D0E94032859
:102C2000D70114968D919C9115978A0D9B1D159631
:102C30009C938E931497ED91FC911197E80FF91FD7
:102C400010822D913C912C0F3D1FF6016081718106
:102C500044815581C9010E94FA279E0105C0D70110
:102C600014962D913C9115972150304037FFBACFE3
:102C7000DF91CF911F910F91FF90EF90DF90CF9058
:102C8000BF90AF909F908F907F906F905F904F908C
:102C90003F902F900895CF93DF93FC01C081D181A5
:102CA000209739F409C0992787FD90950E94DD2768
:102CB000899388818823B9F7DF91CF910895CF93C5
:102CC000DF93FC01C081D181209739F409C0992795
:102CD00087FD90950E94E527899388818823B9F71D
:102CE000DF91CF910895AF92BF92CF92DF92EF9292
:102CF000FF920F931F93CF93DF936C01DC01ED9054
:102D0000FC901197E114F10409F443C01496AD90BE
:102D1000BC901597A114B104E1F18701E801888105
:102D20000F5F1F4F992787FD90950E94D527009729
:102D3000A9F78501015010400E0D1F1DF80180817B
:102D4000992787FD90950E94D527009731F00C17A1
:102D50001D0718F001501040F1CF0F5F1F4F0C1BE3
:102D60001D0BD60115961C930E931497EC16FD06B9
:102D700028F4C701BE01A8010E94FA27D601ED91EF
:102D8000FC91119714968D919C911597E80FF91F5E
:102D90001082DF91CF911F910F91FF90EF90DF9004
:102DA000CF90BF90AF900895FC01808191810097F2
:102DB00029F00E94AE279B01AC0103C020E030E067
:102DC000A901B901CA0108950E945B2508950E94D6
:102DD000F525089521E030E0FC018081882311F081
:102DE00020E030E0C901089521E0FC01208308952E
:102DF000089508951F920F920FB60F9211242F93EA
:102E00003F934F935F936F937F938F939F93AF9372
:102E1000BF932091C5033091C6034091C7035091E1
:102E2000C8037091C903DA01C9010296A11DB11D41
:102E3000672F6A5F6D3730F06D57DA01C90103966D
:102E4000A11DB11D6093C9038093C5039093C60370
:102E5000A093C703B093C8038091C1039091C203AC
:102E6000A091C303B091C4030196A11DB11D80932D
:102E7000C1039093C203A093C303B093C403BF9153
:102E8000AF919F918F917F916F915F914F913F9102
:102E90002F910F900FBE0F901F9018958FB7F89439
:102EA0002091C5033091C6034091C7035091C803D8
:102EB0008FBFB901CA0108959FB7F8942091C1034B
:102EC0003091C2034091C3035091C40386B5A89BBF
:102ED00006C08F3F21F02F5F3F4F4F4F5F4F9FBF87
:102EE000542F432F322F2227280F311D411D511DF2
:102EF00083E0220F331F441F551F8A95D1F7B90174
:102F0000CA010895EF92FF920F931F93CF93DF931F
:102F10007B018C010E945C17EB010FC00E945C17C3
:102F20006C1B7D0B83E0683E780738F00894E1085D
:102F3000F10801091109C851DC4FE114F104010540
:102F4000110561F7DF91CF911F910F91FF90EF90E5
:102F50000895019739F0019729F0880F991F01977B
:102F60000197F1F70895789484B5826084BD84B5A3
:102F7000816084BD85B5826085BD85B5816085BD74
:102F8000EEE6F0E0808181608083E1E8F0E010828D
:102F9000808182608083808181608083E0E8F0E0CE
:102FA000808181608083E1EBF0E0808184608083B8
:102FB000E0EBF0E0808181608083EAE7F0E08081EF
:102FC000846080838081826080838081816080834F
:102FD0008081806880831092C10008958093AD0144
:102FE00008958E3008F08E5087709091AD019295C3
:102FF000990F990F907C982B90937C0080917A0088
:10300000806480937A0080917A0086FDFCCF2091C5
:10301000780030917900932F80E030E0282B392B15
:10302000C90108951F93CF93DF93182FEB0161E03F
:103030000E949F18209709F44AC0CF3FD10509F498
:1030400049C0E12FF0E0E155FF4FE491E330C1F0DA
:10305000E43028F4E13051F0E230B1F50CC0E63054
:1030600019F1E73049F1E43079F514C084B580688E
:1030700084BDC7BD33C084B5806284BDC8BD2EC0C9
:1030800080918000806880938000D0938900C093F5
:10309000880024C080918000806280938000D0935B
:1030A0008B00C0938A001AC08091B0008068809322
:1030B000B000C093B30012C08091B00080628093D2
:1030C000B000C093B4000AC0C038D1051CF4812FF1
:1030D00060E002C0812F61E00E94C318DF91CF91B0
:1030E0001F910895833071F0843028F48130A1F06D
:1030F000823021F514C08630B1F08730D1F08430B1
:10310000E9F404C0809180008F7703C08091800033
:103110008F7D80938000089584B58F7702C084B539
:103120008F7D84BD08958091B0008F778093B0002B
:1031300008958091B0008F7D8093B000089590E055
:10314000FC01E556FF4F2491FC01E957FF4FE49144
:10315000EE23C1F0F0E0EE0FFF1FE759FF4F85911E
:103160009491DC01662341F49FB7F8948C912095EB
:1031700082238C939FBF08959FB7F8948C91822BE4
:103180008C939FBF08950F931F93DF93CF930F925C
:10319000CDB7DEB7282F30E0F901E155FF4F84911C
:1031A000F901E556FF4F149129573F4FF90104915A
:1031B0000023D9F0882321F069830E947218698165
:1031C000E02FF0E0EE0FFF1FED58FF4F8591949137
:1031D000DC019FB7F894662321F48C91109581232C
:1031E00002C08C91812B8C939FBF0F90CF91DF9168
:1031F0001F910F9108950F931F93282F30E0F9012D
:10320000E155FF4F8491F901E556FF4F049129578D
:103210003F4FF9011491112391F0882311F00E947E
:103220007218E12FF0E0EE0FFF1FE358FF4F85917A
:103230009491DC018C91802321E030E011F420E0B6
:1032400030E0C9011F910F9108958F929F92AF9224
:10325000BF92CF92DF92EF92FF920F931F9390E075
:10326000FC01E556FF4F949089579F4FFC01E49075
:10327000662311F4882401C0892CCA01B90120E415
:103280003FE140E050E00E949B2420E83EE340E024
:1032900050E00E94CD2459016A0180E090E0DC01F9
:1032A0006E2D70E0FB01EE0FFF1FE358FF4F2591DD
:1032B000349109C08A159B05AC05BD0509F44DC0C4
:1032C0000196A11DB11DF90140814921481591F3D5
:1032D0000AC08A159B05AC05BD0509F43EC00196E0
:1032E000A11DB11D07C0660F771F63587F4FFB01FB
:1032F00025913491F90140814921481551F720E089
:1033000030E0A901FB01659174910FC079018A0138
:10331000E80EF91E0A1F1B1FEA14FB040C051D050D
:10332000E1F02F5F3F4F4F4F5F4FFB01E081E921FD
:10333000E81561F3CA01B90128E032E540E050E048
:103340000E949B246058714C8F4F9F4F20E43FE1B7
:1033500040E050E00E94CD2403C020E030E0A9010D
:10336000B901CA011F910F91FF90EF90DF90CF90AC
:10337000BF90AF909F908F900895CF92DF92EF9281
:10338000FF920F931F93CF93DF93E82EF62EC42E58
:10339000C7E0D0E0DD2407E010E08F2D61E00E945F
:1033A000C318CC2071F48E2D0E94FB1898012C1BA1
:1033B0003D0BAC0102C0440F551F2A95E2F79A015C
:1033C0000AC08E2D0E94FB189C010C2E02C0220FF9
:1033D000331F0A94E2F7D22A8F2D60E00E94C318AF
:1033E00021975FEFCF3FD507C1F68D2DDF91CF91AC
:1033F0001F910F91FF90EF90DF90CF900895BF92B3
:10340000CF92DF92EF92FF920F931F93CF93DF93B0
:10341000C82ED62EB42EC7E0D0E0022F10E087E0F1
:10342000E82EF12CBB2059F497012C1B3D0BC80151
:1034300002C0959587952A95E2F79C0107C09801EF
:103440000C2E02C0359527950A94E2F7622F617021
:103450008C2D0E94C3188D2D61E00E94C3188D2D04
:1034600060E00E94C31821979FEFCF3FD907D1F6A4
:10347000DF91CF911F910F91FF90EF90DF90CF9050
:10348000BF9008952091EB0330E08091EA03281B60
:103490003109C90108958091EA039091EB038917DE
:1034A00050F4E82FF0E0E653FC4F208130E08F5FCE
:1034B0008093EA0302C02FEF3FEFC9010895E09126
:1034C000EA038091EB03E81730F4F0E0E653FC4F99
:1034D000208130E002C02FEF3FEFC9010895089529
:1034E000CF93DF939C01CB01E0911204F091130480
:1034F0003097D9F05091EA034091EB035417A8F0AC
:1035000060E009C0DA01A653BC4F420F531FEA0125
:1035100048814C936F5F462F50E04817590794F34A
:103520001092EA038093EB030995DF91CF91089500
:10353000E0911004F0911104309729F010920D04DD
:1035400010920E0409950895CF92DF92EF92FF92A8
:103550000F931F93CF93DF936C01CB01EA0120916E
:103560000F042223B1F0E62EF92E00E010E00DC08A
:10357000D7016D917D01D601ED91FC910190F08113
:10358000E02DC60109950F5F1F4F0C171D0780F333
:1035900003C0642F0E94191CCE01DF91CF911F91AF
:1035A0000F91FF90EF90DF90CF900895DF93CF932E
:1035B0000F92CDB7DEB7698320910F042223D1F09B
:1035C00020910E04203240F021E030E0FC013383F2
:1035D000228320E030E015C080910D04E82FF0E058
:1035E000E351FC4F998190838F5F80930D0480930A
:1035F0000E0405C0CE01019661E00E94191C21E075
:1036000030E0C9010F90CF91DF910895FC01138242
:10361000128228EE33E040E050E024833583468375
:10362000578382EB91E09183808308951092EA039F
:103630001092EB0310920D0410920E040E94861B50
:103640000895CF93DF93EC01862F0E949F1B88E99A
:103650009AE10E94381C80E79AE10E94331CCE0157
:103660000E94161BDF91CF9108950E94211B08959F
:10367000862F413208F040E26AEC73E00E94A31BFF
:103680001092EA038093EB0308950E94381B08957B
:1036900081E080930F046093EC0310920D0410926C
:1036A0000E0408950E94481B08958091EC036DEE6E
:1036B00073E040910E0421E00E94D91B10920D048A
:1036C00010920E0410920F040895709313046093E7
:1036D00012040895709311046093100408951092D9
:1036E00017041092160488EE93E0A0E0B0E08093F7
:1036F000180490931904A0931A04B0931B0482EB4E
:1037000091E090931504809314040895109244045A
:1037100082E161E00E94C31883E161E00E94C31866
:10372000E9EBF0E080818E7F808380818D7F8083D4
:1037300080E28093B80085E48093BC000895880FF0
:103740008093BA000895413288F5909144049923FA
:10375000E1F791E0909344049FEF9093430410921B
:103760002104942F915090932204880F81608093BC
:10377000200485EE8093BC00809144048130E1F305
:1037800080912104841710F440912104E3E2F4E0D5
:10379000262F372FD901242F30E02E0F3F1F02C0D4
:1037A00081918D93E217F307D9F701C040E0842F90
:1037B00008954132B0F5909144049923E1F792E0E5
:1037C000909344049FEF90934304109221044093FC
:1037D0002204DB01E3E2F4E050E04E0F5F1F02C081
:1037E0009D919193E417F507D9F790E0880F991F01
:1037F0008093200485EE8093BC00222321F08091E9
:1038000044048230E1F3809143048F3F61F0809162
:103810004304803251F080914304803341F483E0CB
:10382000089581E0089580E0089582E0089584E09D
:1038300008956132A0F420914404243091F46093FF
:103840006904DC01ECE6F4E070E06E0F7F1F02C05B
:103850008D918193E617F707D9F780E0089581E00D
:10386000089582E008959093670480936604089514
:1038700090936B0480936A040895882311F085EC7B
:1038800001C085E88093BC00089585ED8093BC005D
:103890008091BC0084FDFCCF10924404089585EC17
:1038A0008093BC001092440408951F920F920FB6AB
:1038B0000F9211242F933F934F935F936F937F93B6
:1038C0008F939F93AF93BF93EF93FF938091B90032
:1038D00090E0887F90708036910509F4C2C08136EF
:1038E0009105E4F58832910509F47EC0893291058D
:1038F000C4F48031910509F472C08131910544F41A
:10390000009709F413C18830910509F013C167C00D
:103910008831910509F468C08032910509F00AC127
:1039200078C08034910509F48AC0813491054CF443
:103930008033910509F46FC08833910509F0FAC00E
:103940006EC08035910509F46EC08835910509F483
:103950007BC08834910509F0EDC0EAC08839910533
:1039600009F4DAC089399105ECF48837910509F436
:1039700078C0893791054CF48836910509F471C0F7
:103980008037910509F0D6C06CC08838910509F4DC
:10399000C3C08039910509F46AC08038910509F0E7
:1039A000C9C065C0803B910509F48EC0813B91057B
:1039B0004CF4803A910509F46CC0883A910509F0FD
:1039C000B9C082C0803C910509F4AAC0883C910529
:1039D00009F4A6C0883B910509F0ACC08AC080916B
:1039E00020048093BB0013C0909121048091220495
:1039F000981708F09DC080912104E82FF0E0ED5D5C
:103A0000FB4F90819093BB008F5F8093210481E0F6
:103A100084C080E201C080E38093430489C088E3CE
:103A2000809343044EC0809121049091BB00E82F05
:103A3000F0E0ED5DFB4F90838F5F809321049091C8
:103A400021048091220465C0809121049091BB00E3
:103A5000E82FF0E0ED5DFB4F90838F5F80932104B2
:103A600067C083E08093440410924504D0CF8091D6
:103A70004504803208F050C0809145049091BB000D
:103A8000E82FF0E0EA5BFB4F90838F5F8093450463
:103A9000BECF80914504803230F4E0914504F0E0DF
:103AA000EA5BFB4F10820E94451C60914504E09147
:103AB0006604F091670486E494E070E00995109242
:103AC00045040E944F1C36C084E080934404109249
:103AD000680410926904E0916A04F0916B040995FE
:103AE00080916904882329F481E08093690410920D
:103AF0006C0480916804E82FF0E0E459FB4F90815A
:103B00009093BB008F5F80936804909168048091CC
:103B10006904981708F47BCF80E00E943D1C0AC01E
:103B200081E00E943D1C1092440404C010924304A2
:103B30000E94451CFF91EF91BF91AF919F918F9192
:103B40007F916F915F914F913F912F910F900FBE99
:103B50000F901F901895EF92FF920F931F937B0188
:103B60008C0120E030E040E05FE40E94272187FDE7
:103B700011C0C801B70120E030E040E05FE40E94DE
:103B80004E1F0E94E7219B01AC0120503040404075
:103B9000504806C0C801B7010E94E7219B01AC0153
:103BA000B901CA011F910F91FF90EF900895A0E015
:103BB000B0E0EDEDFDE10C942225FC01EA018081ED
:103BC000823008F438C1DB019C91923008F430C196
:103BD000843059F4943009F02EC1918111968C9162
:103BE0001197981709F021C126C1943009F420C11A
:103BF0009230B1F4823009F01EC1CA01AF0128E051
:103C0000DA010D90AD01DC010D92CD012150C1F71B
:103C1000DB0111968C9111979181892389830AC1C7
:103C2000823009F405C1C280D380DB0112966D9009
:103C30007C90139724813581468157811496ED90AD
:103C4000FD900D911C911797C601861997095C018B
:103C500097FF04C0AA24BB24A81AB90AB0E2AB1685
:103C6000B1040CF061C0181619066CF53701480153
:103C70000A2C04C096948794779467940A94D2F798
:103C800081E090E0A0E0B0E00A2C04C0880F991F0A
:103C9000AA1FBB1F0A94D2F70197A109B1098E216F
:103CA0009F21A023B123EE24FF248701E3940097F2
:103CB000A105B10519F4EE24FF248701E628F728B1
:103CC000082919293CC00097D1F1CA0CDB1C390125
:103CD0004A010A2C04C096948794779467940A94B6
:103CE000D2F781E090E0A0E0B0E00A2C04C0880F99
:103CF000991FAA1FBB1F0A94D2F70197A109B10906
:103D000082239323A423B52321E030E040E050E058
:103D10000097A105B10519F420E030E0A90126299A
:103D20003729482959290BC06C147D0424F4EE244A
:103D3000FF24870104C0630120E030E0A9018181F4
:103D4000FB019181891709F445C0882349F0D80106
:103D5000C701821B930BA40BB50B9C01AD0104C0E2
:103D60002E193F09400B510B57FD04C01982DB820D
:103D7000CA820BC081E08983DB82CA82509540955C
:103D8000309521953F4F4F4F5F4F2C833D834E839E
:103D90005F830DC0880F991FAA1FBB1F8C839D8353
:103DA000AE83BF838A819B8101979B838A838C81A9
:103DB0009D81AE81BF819C01AD01215030404040CA
:103DC00050402F3FEFEF3E07EFEF4E07EFE35E0768
:103DD00008F30BC08983DB82CA822E0D3F1D401F72
:103DE000511F2C833D834E835F8383E088832C8126
:103DF0003D814E815F8157FF1DC0DA01C90181708D
:103E00009070A070B0705695479537952795822B86
:103E1000932BA42BB52B8C839D83AE83BF838A8188
:103E20009B8101969B838A8305C0EEECF1E003C081
:103E3000FB0101C0FE01CF01CDB7DEB7EEE00C946F
:103E40003E25A0E2B0E0E7E2FFE10C942A25698379
:103E50007A838B839C832D833E834F83588789E0AD
:103E6000E82EF12CEC0EFD1ECE010196B7010E944A
:103E7000D9238E010F5E1F4FCE010596B8010E9417
:103E8000D923C701B801AE01475E5F4F0E94D71D1D
:103E90000E940B23A096E6E00C944625A0E2B0E039
:103EA000E4E5FFE10C942A2569837A838B839C8364
:103EB0002D833E834F8358878E01075F1F4FCE01AE
:103EC0000196B8010E94D92391E1E92EF12CEC0E64
:103ED000FD1ECE010596B7010E94D9238A8991E083
:103EE00089278A8BC801B701AE01475E5F4F0E94E8
:103EF000D71D0E940B23A096E6E00C944625A0E275
:103F0000B0E0E5E8FFE10C941E2569837A838B839A
:103F10009C832D833E834F835887CE010196BE013B
:103F2000675F7F4F0E94D923CE010596BE016F5E69
:103F30007F4F0E94D9239985923078F08989823009
:103F4000C0F0943019F4823041F4CBC0843019F4BD
:103F5000923079F4C6C0923051F481E02A859A8972
:103F6000291709F480E08A87CE010996BCC0823007
:103F700051F481E02A859A89291709F480E08A8B17
:103F8000CE014196B0C06D847E848F849888ED8880
:103F9000FE880F89188DE0E2F0E080E090E0DC011F
:103FA000AA24BB24650120E030E0A901B3016170BF
:103FB000707061157105D1F02E0D3F1D401F511F0E
:103FC00015012601280E391E4A1E5B1E81E090E075
:103FD000A0E0B0E02E153F054007510718F080E043
:103FE00090E0DC01820D931DA41DB51DAA0CBB1C25
:103FF000CC1CDD1C17FF09C061E0262E312C412CA2
:10400000512CA228B328C428D528319749F0EE0CAA
:10401000FF1C001F111F9694879477946794C6CF56
:104020006B897C89EB85FC856E0F7F1F6E5F7F4FF0
:104030007C8F6B8F61E0EA857A89E71709F460E08D
:104040006A8F6B8D7C8D10C0FC01E170F070309731
:1040500029F056954795379527955068B695A795B9
:10406000979587956F5F7F4FB7FDEECF0CC0880F98
:10407000991FAA1FBB1F57FD8160220F331F441FCA
:10408000551F615070408030E0E09E07E0E0AE07D1
:10409000E0E4BE0760F36B8F7C8F6FE7E62EF12CB8
:1040A000012D112DE822F9220A231B2360E4E616D4
:1040B000F1040105110561F487FD0AC021153105E0
:1040C0004105510529F0805C9F4FAF4FBF4F80786D
:1040D0008D8F9E8FAF8FB8A383E0898FCE014996D5
:1040E00002C08EEC91E00E940B23A096E2E10C94BA
:1040F0003A25A8E1B0E0EFE7F0E20C9426256983C9
:104100007A838B839C832D833E834F8358878E01D4
:10411000075F1F4FCE010196B8010E94D92381E1AC
:10412000E82EF12CEC0EFD1ECE010596B7010E9483
:10413000D9239985923008F483C08989823008F4A4
:104140007BC02A853A8923272A87943011F0923040
:1041500021F4981709F06CC071C0843039F41D86C1
:104160001E861F86188A1C861B866AC0823019F438
:1041700084E0898765C08B859C852B893C89821B5F
:10418000930B9C878B872D853E854F855889ED88BD
:10419000FE880F89188D2E153F054007510738F40A
:1041A000220F331F441F551F01979C878B876FE198
:1041B00070E0A12CB12CC12CA0E4DA2E80E090E0BC
:1041C000DC012E153F054007510740F08A299B2945
:1041D000AC29BD292E193F09400B510BD694C79429
:1041E000B794A794220F331F441F551F615070408E
:1041F00041F76FE7E62EF12C012D112DE822F9226F
:104200000A231B2360E4E616F1040105110561F49D
:1042100087FD0AC0211531054105510529F0805C53
:104220009F4FAF4FBF4F80788D879E87AF87B88BEA
:104230008E01075F1F4F04C0870102C00EEC11E022
:10424000C8010E940B236896EAE00C944225A8E17D
:10425000B0E0EDE2F1E20C942A2569837A838B8346
:104260009C832D833E834F8358878E01075F1F4FAA
:10427000CE010196B8010E94D92381E1E82EF12CEC
:10428000EC0EFD1ECE010596B7010E94D92389854B
:10429000823040F08989823028F0C801B7010E943D
:1042A000422401C08FEF6896E6E00C944625A8E111
:1042B000B0E0EDE5F1E20C942A2569837A838B83E3
:1042C0009C832D833E834F8358878E01075F1F4F4A
:1042D000CE010196B8010E94D92381E1E82EF12C8C
:1042E000EC0EFD1ECE010596B7010E94D9238985EB
:1042F000823040F08989823028F0C801B7010E94DD
:10430000422401C081E06896E6E00C944625A8E0CE
:10431000B0E0EDE8F1E20C942A257B018C0183E00A
:104320008983D801C7018827B7FD83959927AA27D4
:10433000BB27282F8A83E114F1040105110519F424
:1043400082E0898337C08EE190E09C838B832223B7
:1043500089F080E0E81680E0F80680E0080780E851
:10436000180769F110950095F094E094E11CF11C98
:10437000011D111DED82FE820F831887C801B70150
:104380000E94B1229C01215030401216130694F471
:10439000022E04C0EE0CFF1C001F111F0A94D2F75E
:1043A000ED82FE820F8318878EE190E0821B930BD3
:1043B0009C838B83CE0101960E940B2304C060E096
:1043C00070E080E09FEC2896E6E00C944625ACE097
:1043D000B0E0EDEEF1E20C942E2569837A838B83B5
:1043E0009C83CE010196BE016B5F7F4F0E94D92353
:1043F0008D81823081F1823070F1843021F48E81A0
:10440000882369F10AC02F81388537FD24C06E8169
:104410002F3131053CF0662311F120E030E040E01F
:1044200050E821C08EE190E0821B930B29853A85EC
:104430004B855C8504C056954795379527958A9599
:10444000D2F7662381F050954095309521953F4FE6
:104450004F4F5F4F08C020E030E0A90104C02FEFAC
:104460003FEF4FEF5FE7B901CA012C96E2E00C94F1
:104470004A25A8E0B0E0EFE3F2E20C9428257B01A6
:104480008C011A82611571058105910519F482E08C
:1044900089835FC083E089838EE1C82ED12CDC82C2
:1044A000CB82ED82FE820F831887C801B7010E947C
:1044B000B122FC013197F7FF3AC0AA27BB27AE1BF8
:1044C000BF0B21E030E040E050E00A2E04C0220F94
:1044D000331F441F551F0A94D2F7215030404040EB
:1044E00050402E213F214023512361E070E080E0C5
:1044F00090E0211531054105510519F460E070E0A7
:10450000CB0104C016950795F794E794AA95D2F7C6
:10451000E62AF72A082B192BED82FE820F831887D3
:104520008EE190E08E1B9F0B9C838B8312C0309793
:1045300081F00E2E04C0EE0CFF1C001F111F0A9408
:10454000D2F7ED82FE820F831887CE1ADF0ADC8253
:10455000CB82CE0101960E940B232896E8E00C94B2
:104560004425AF92BF92CF92DF92EF92FF920F93CA
:104570001F937B018C0180E0E81680E0F80681E063
:10458000080780E0180758F4EFEFEE16F104010574
:10459000110509F090F480E090E0DC0117C0F0E034
:1045A000EF16F0E0FF06F0E00F07F1E01F0750F410
:1045B00080E190E0A0E0B0E009C088E090E0A0E0F9
:1045C000B0E004C088E190E0A0E0B0E020E230E09C
:1045D00040E050E0281B390B4A0B5B0B5701680188
:1045E00004C0D694C794B794A7948A95D2F7D601FD
:1045F000C5018A529E4FFC018081281B3109410967
:104600005109C9011F910F91FF90EF90DF90CF905A
:10461000BF90AF900895EF92FF920F931F93CF93A7
:10462000DF93FC012481358146815781618180813E
:10463000823020F44061EFEFF0E0A3C0843009F451
:104640009BC0823009F492C0211531054105510506
:1046500009F48FC00280F381E02D8FEFE238F80774
:104660000CF05AC0C2E8DFEFCE1BDF0BCA31D10518
:104670006CF579018A010C2E04C016950795F79404
:10468000E7940A94D2F781E090E0A0E0B0E00C2E2D
:1046900004C0880F991FAA1FBB1F0A94D2F7019765
:1046A000A109B10982239323A423B52321E030E09B
:1046B00040E050E00097A105B10519F420E030E09A
:1046C000A9012E293F29402B512B03C020E030E0C7
:1046D000A901DA01C9018F779070A070B0708034A1
:1046E0009105A105B10539F427FF09C0205C3F4FB2
:1046F0004F4F5F4F04C0215C3F4F4F4F5F4FE1E092
:10470000F0E0203080E0380780E0480780E4580778
:1047100028F5E0E0F0E022C0E038F1056CF5E15862
:10472000FF4FDA01C9018F779070A070B0708034AC
:104730009105A105B10539F427FF09C0205C3F4F61
:104740004F4F5F4F04C0215C3F4F4F4F5F4F57FFAC
:1047500005C05695479537952795319687E056952C
:104760004795379527958A95D1F70BC0E0E0F0E0A3
:1047700005C0E0E0F0E005C0EFEFF0E020E030E061
:10478000A9018E2F879588278795942F9F77679506
:1047900066276795E695E22EA92FA82BFE2FF62B0C
:1047A000622F732F8A2F9F2FCDB7DEB7E6E00C94D0
:1047B0004625DC01FB012C9111963C911197129634
:1047C0008C911297482F4F7750E0982F991F992777
:1047D000991F13966C911397862F880F892B90E061
:1047E000661F6627661F6183009739F5211531051D
:1047F0004105510511F482E029C082E89FEF9383BF
:10480000828367E0220F331F441F551F6A95D1F73B
:1048100083E0808309C0220F331F441F551F82810C
:104820009381019793838283203080E0380780E072
:10483000480780E4580778F320C08F3F910579F44A
:10484000211531054105510519F484E0808308954F
:1048500044FF03C081E0808310C010820EC08F57D8
:1048600090409383828383E0808387E0220F331F0D
:10487000441F551F8A95D1F750642483358346839E
:1048800057830895FC01DB019081923008F449C000
:104890008C91823008F445C0943051F461818430A9
:1048A000B1F511962C91119730E0261B310941C0CA
:1048B000843021F0923041F48230B1F111968C9124
:1048C00011978823A1F12DC06181823001F11196E9
:1048D0008C9111976817D9F42281338112968D91AA
:1048E0009C9113978217930794F028173907BCF00F
:1048F000248135814681578114968D919D910D902B
:10490000BC91A02D82179307A407B50718F466235E
:1049100041F00DC0281739074A075B0728F46623C2
:1049200031F021E030E005C020E030E002C02FEFA0
:104930003FEFC9010895629FD001739FF001829FEC
:10494000E00DF11D649FE00DF11D929FF00D839F1E
:10495000F00D749FF00D659FF00D9927729FB00DBB
:10496000E11DF91F639FB00DE11DF91FBD01CF01CE
:104970001124089597FB092E07260AD077FD04D04D
:1049800049D006D000201AF4709561957F4F0895A4
:10499000F6F7909581959F4F0895A1E21A2EAA1BD4
:1049A000BB1BFD010DC0AA1FBB1FEE1FFF1FA217DF
:1049B000B307E407F50720F0A21BB30BE40BF50BDC
:1049C000661F771F881F991F1A9469F76095709565
:1049D000809590959B01AC01BD01CF01089597FB97
:1049E000092E05260ED057FD04D0D7DF0AD0001CB3
:1049F00038F450954095309521953F4F4F4F5F4F7C
:104A00000895F6F790958095709561957F4F8F4F3B
:104A10009F4F0895AA1BBB1B51E107C0AA1FBB1FD4
:104A2000A617B70710F0A61BB70B881F991F5A953A
:104A3000A9F780959095BC01CD0108952F923F92E2
:104A40004F925F926F927F928F929F92AF92BF929E
:104A5000CF92DF92EF92FF920F931F93CF93DF934A
:104A6000CDB7DEB7CA1BDB0B0FB6F894DEBF0FBEA7
:104A7000CDBF09942A88398848885F846E847D84F4
:104A80008C849B84AA84B984C884DF80EE80FD80F6
:104A90000C811B81AA81B981CE0FD11D0FB6F8946C
:104AA000DEBF0FBECDBFED010895EE0FFF1F0590D5
:104AB000F491E02D0994CF93DF938230910510F4A7
:104AC00082E090E0E0918E04F0918F0440E050E0AD
:104AD00020E030E026C06081718168177907E0F03E
:104AE0006817790781F4828193812115310531F0AE
:104AF000D90113969C938E9312972BC090938F0499
:104B000080938E0426C04115510519F0641775076E
:104B100018F4AB01E901DF019F0172816381E72F86
:104B2000F62F3097C1F64115510501F1481B590B7D
:104B30004430510580F412968D919C9113972097E3
:104B400019F09B838A8304C090938F0480938E0412
:104B5000FD01329646C0FD01E40FF51F819391934C
:104B60004250504011965C934E933BC020918C0470
:104B700030918D042115310541F42091D8023091F6
:104B8000D90230938D0420938C042091DA02309165
:104B9000DB022115310541F42DB73EB74091D60215
:104BA0005091D702241B350BE0918C04F0918D04B9
:104BB000E217F307A0F42E1B3F0B2817390778F0F4
:104BC000AC014E5F5F4F2417350748F04E0F5F1F53
:104BD00050938D0440938C048193919302C0E0E044
:104BE000F0E0CF01DF91CF910895CF93DF9300974D
:104BF00009F491C0FC0132971382128260918E04F5
:104C000070918F046115710581F420813181280F25
:104C1000391F80918C0490918D048217930799F528
:104C2000F0938D04E0938C0476C0DB0180E090E08B
:104C300002C0CD01D901AE17BF0748F412962D91DD
:104C40003C91139721153105A1F7CD0121C0B38304
:104C5000A283EF01499159919E01240F351FA2179C
:104C6000B30779F42D913C911197240F351F2E5FD6
:104C70003F4F3183208312962D913C9113973383BC
:104C80002283009729F4F0938F04E0938E0443C0AD
:104C9000DC011396FC93EE9312974D915D91A40F56
:104CA000B51FEA17FB0769F420813181240F351FF6
:104CB0002E5F3F4FEC0139832883228133813B8370
:104CC0002A83E0E0F0E002C0FB01BC01DB011296A8
:104CD0008D919C9113970097B9F79B012E5F3F4FE1
:104CE0008D919C911197820F931F40918C0450914C
:104CF0008D044817590779F4309729F410928F04DE
:104D000010928E0402C013821282225030403093DF
:104D10008D0420938C04DF91CF910895A0E0B0E042
:104D2000E4E9F6E20C942625EC01688179818A8118
:104D30009B81611571058105910521F464E279ED8E
:104D40008BE597E02DE133EF41E050E00E94EF2446
:104D500079018A0127EA31E440E050E00E949B2477
:104D60005B016C01C801B7012CEE34EF4FEF5FEF30
:104D70000E949B249B01AC012A0D3B1D4C1D5D1D17
:104D800057FF04C0215030404040504828833983A9
:104D90004A835B835F77B901CA01CDB7DEB7EAE02A
:104DA0000C9442250E948E2608958CED92E00E947C
:104DB0008E2608956093DC027093DD028093DE02FC
:104DC0009093DF020895A0E0B0E0E9EEF6E20C94E3
:104DD00024258C01CB010115110529F40E945B25C6
:104DE000082F192FB5C0D80112979801260F371F29
:104DF0002A173B0708F4AAC0ED90FC901197E6161D
:104E0000F706D0F045E0E416F10408F4A1C0A701CC
:104E1000445050404617570708F49AC0A701425023
:104E20005040461B570BF901419351936D937C936E
:104E3000CF010E94F5258CC05B01AE18BF08480168
:104E40008E0C9F1CE0918E04F0918F04CC24DD2405
:104E5000C0E0D0E041C0E815F90599F560817181A5
:104E6000AB014E5F5F4F4A155B0558F1AB014A1924
:104E70005B09CC24DD246894C1F8C40ED51E828061
:104E8000A380E5E0CE16D10448F0F9018282A38226
:104E90005183408311969C938E9309C0C70102965B
:104EA000860F971F11969C938E93E82DFA2D2097CD
:104EB00019F0FB83EA834CC0F0938F04E0938E04D7
:104EC00047C040815181C416D50608F46A01EF013C
:104ED00052814381E52FF42F309709F0BCCF4091E8
:104EE0008C0450918D0448155905E9F4C816D9066B
:104EF000D0F44091DA025091DB024115510541F4A2
:104F00004DB75EB76091D6027091D702461B570B22
:104F100024173507D8F430938D0420938C04119610
:104F20009C938E9315C00E945B25C82EE6016E01EE
:104F3000D92EE601209751F08C2DB801A7010E94CF
:104F4000FA27C8010E94F525860102C000E010E0A2
:104F5000C801CDB7DEB7ECE00C9440251F93FC01EF
:104F600099278827BC01E89411911032E9F3193090
:104F700010F01E30C8F31B3251F01D3249F4689412
:104F800006C00E94C728610F711D811D911D1191DE
:104F900010531A30B0F33EF490958095709561955A
:104FA0007F4F8F4F9F4F1F910895911140C18032C5
:104FB00019F089508550D0F70895911108958154C2
:104FC0008A5108F4805E855A08959111089581569A
:104FD0008A5108F4805285580895FB01DC0104C011
:104FE0008D910190801921F441505040C8F7881BE1
:104FF000990B0895FB01DC0102C001900D92415014
:105000005040D8F708956817790768F4FB01DC0170
:10501000E40FF51FA40FB51F02C002900E9241507D
:105020005040D8F708950C94FA27FC018191861717
:1050300021F08823D9F7992708953197CF01089552
:10504000FB01DC018D91019080190110D9F3990BBE
:105050000895FB01DC0101900D920020E1F7089515
:10506000FB01DC014150504030F08D9101908019DE
:1050700019F40020B9F7881B990B0895FB01DC0196
:105080004150504048F001900D920020C9F701C0F6
:105090001D9241505040E0F70895FC0181E090E0FE
:1050A0000190061609F4CF010020D1F70197089569
:1050B000FB0151915523A9F0BF01DC014D9145172A
:1050C0004111E1F759F4CD010190002049F04D91D3
:1050D00040154111C9F3FB014111EFCF81E090E090
:1050E00001970895FB019F01E8944230C4F04532D6
:1050F000B4F44A3029F497FB1EF4909581959F4FA4
:10510000642F77270E940A25805D8A330CF0895D21
:105110008193CB010097A1F716F45DE251931082C1
:10512000C9010C941A29FA01CF93FF93EF9322300F
:1051300044F1253234F5C22FE894CA3049F497FB84
:105140003EF490958095709561957F4F8F4F9F4F5E
:105150002C2F332744275527FF93EF930E94CD240C
:10516000EF91FF91605D6A330CF0695D6193B90165
:10517000CA01605070408040904051F716F4CDE273
:10518000C19310828F919F91CF910C941A29592F1E
:10519000482F372F262F660F771F881F991F660FFE
:1051A000771F881F991F620F731F841F951F660F3B
:1051B000771F881F991F0895FA01CF93FF93EF93EC
:1051C0002230CCF02532BCF4C22F2C2F33274427B9
:1051D0005527FF93EF930E94CD24EF91FF91605DDF
:1051E0006A330CF0695D6193B901CA016050704087
:1051F0008040904051F710828F919F91CF910C94F5
:105200001A29FB019F01423074F0453264F4642F87
:1052100077270E940A25805D8A330CF0895D81938F
:10522000CB010097A1F71082C9010C941A29992784
:1052300088270895DC01FC01672F71917723E1F73E
:10524000329704C07C916D9370836291AE17BF0753
:08525000C8F30895F894FFCFA4
:105258000D0A2B494E513D310D0A000D0A2B5354AE
:10526800574D4F443D300D0A000D0A2B53544E4103
:105278003D4164617074696373456C656374696307
:105288000D0A000D0A2B53544F4155543D310D0A58
:10529800000D0A2B53544155544F3D300D0A000D53
:1052A8000A202B535450494E3D303030300D0A00FF
:1052B8000D0A2B4C4F53535245434F4E4E3D300D24
:1052C8000A0007F00000000000B00286054B027AD1
:1052D800025E029C0200000000F9168605F916F924
:1052E80016F916F91600000000DE0400000000F9A7
:1052F800162E0000000000F9168605FF00010000C8
:105308000000D61AA41A421A4B1A5F1A6F1A000024
:105318000000F9168605F916F916F916F9160000AF
:10532800000000000000000102020303030304045C
:10533800040404040404050505050505050505051B
:1053480005050505050506060606060606060606FB
:1053580006060606060606060606060606060606E5
:1053680006060606060607070707070707070707CB
:1053780007070707070707070707070707070707B5
:1053880007070707070707070707070707070707A5
:105398000707070707070707070707070707070795
:1053A800070707070707080808080808080808087B
:1053B8000808080808080808080808080808080865
:1053C8000808080808080808080808080808080855
:1053D8000808080808080808080808080808080845
:1053E8000808080808080808080808080808080835
:1053F8000808080808080808080808080808080825
:105408000808080808080808080808080808080814
:105418000808080808080808080808080808080804
:10542800080808080808200090040000010000008F
:00000001FF
